:100000000C9466030C94AD030C94AD030C94AD03F7
:100010000C94AD030C94AD030C94AD030C94AD03A0
:100020000C94AD030C94AD030C94350E0C94070F97
:100030000C94AD030C94AD030C94AD030C94AD0380
:100040000C94AD030C947B230C94AD030C94AD0382
:100050000C94AD030C940D1D0C94AD030C94AD03E6
:100060000C94AD030C94AD030C94AD030C94AD0350
:100070000C94AD030C94AD030C94AD030C94AD0340
:100080000C94AD030C94AD030C94AD030C94AD0330
:100090000C94AD030C94AD030C94AD030C94AD0320
:1000A0000C94AD030C94AD030C94AD03740F960F38
:1000B0008910960F8910DB0FFE0F89105310661000
:1000C000501350137F137F13C213FC130916091624
:1000D000151409160A150A15DD1509160916F41561
:1000E0000122022201C402C4000121022101C40232
:1000F000C4000120022001C402C400011F021F012C
:10010000C402C4000131023101C402C40001E10192
:1001100031023102E101C402C4000126022601C4F9
:1001200002C4000125022501C402C40001240224E6
:1001300001C402C4000123022301C402C40001E17E
:100140000134023402E101C402C400012D022D0178
:10015000C402C40001E10127022702E101C402C474
:100160000001E10125022502E101C402C400011ED3
:10017000021E01C402C40001E10130023002E101AB
:10018000C402C40001E1012F022F02E101C402C434
:10019000000127022701C402C400012E022E01C45F
:1001A00002C40001E10126022602E101C402C400EA
:1001B0000138023801C402C40001E1011E021E021E
:1001C000E101C402C4000130023001C402C40001D4
:1001D0002F022F01C402C40001E1012D022D02E112
:1001E00001C402C40001E10121022102E101C402B3
:1001F000C40001E1011F021F02E101C402C40001A9
:10020000E1012E022E02E101C402C40001E1013825
:10021000023802E101C402C40001E1012402240207
:10022000E101C402C40001E10122022202E101C491
:1002300002C4000000F0A101840884088A35002B64
:1002400000297FE100000000001E00140004001DD2
:100250000000004D001F00070016001B00E0002CEE
:1002600000200015000B001000E2002A0021001AF7
:100270000017000600E3004A00220005000A0019EA
:1002800000000000005000015400000000000000C9
:10029000004F000154000000770000000023000D13
:1002A000001C000E00000000002400090011000FD7
:1002B0000050004B002500180008003600510028AF
:1002C00000260013001200370052002C00270033D4
:1002D000000C0038714F004E002D0031003400E555
:1002E00000C4000000010001000100010001000045
:1002F000003A00220238002300010001003B0024E4
:100300000226022400010001003C0038022E0025D4
:1003100000010001003D002E02270026000100011F
:10032000003E001F022F0231020000010001000107
:1003300000000001000000010001000100000001B8
:1003400000000001003F00210230023800000001DF
:100350000040002D021E001F000100010041002F7F
:100360000025022000010001004200300027022188
:10037000000100010043001E022D002200010001C7
:1003800000440045003400010001000000010001AC
:100390000001000100010000000100010001000156
:1003A000000100010001000100F200010001000154
:1003B000000100F000F1000100F400010001000163
:1003C00000F3000100F5000100010001000100013F
:1003D0000000000100010001000000010000000118
:1003E0000001000100000001000000010001000107
:1003F00000010001000000010001000100010001F6
:1004000000A9000100010001000100AC00AA00B633
:1004100000010001000100AB00A800010001000183
:1004200000010001000100010001000100AE000117
:1004300000010000000100010001000100010000B6
:10044000003A0064306D307830010001003B0065F7
:10045000306E307930010001003C0066306F307A38
:1004600030010001003D00673070307B3001000139
:10047000003E00683071307C300000010001000156
:100480000000000100000001000100010000000167
:1004900000000001003F00693072307D3000000133
:1004A0000040006A3073307E300100010041006B73
:1004B0003074307F300100010042006C30753080B4
:1004C00030010001004300823076308130010001AC
:1004D000004400450077300100010000001603458C
:1004E00000720067006F0044006F00780020004534
:1004F000005A00000016034500720067006F0044B8
:10050000006F007800200045005A00000004030935
:100510000409026D00040100A0FA090400000103AF
:10052000010100092111010001223F00070581039B
:1005300008000A0904010001030102000921110158
:100540000001224D000705820308000A0904020089
:1005500001030000000921110100012236000705F6
:10056000830308000A0904030001030000000921B5
:100570001101000122390007058403100001120156
:10058000100100000008EDFE071301000102000148
:1005900005010906A101050719E029E71500250154
:1005A0009508750181020508190129059505750150
:1005B000910295017503910105071900297715002E
:1005C0002501957875018102C005010980A1018589
:1005D0000216010026B7001A01002AB7007510950F
:1005E000018100C0050C0901A10185031601002647
:1005F0009C021A01002A9C02751095018100C00519
:10060000010902A1010901A1000509190129051526
:10061000002501950575018102950175038101058C
:1006200001093009311581257F9502750881060978
:10063000381581257F950175088106050C0A380259
:100640001581257F950175088106C0C00501090641
:10065000A101050719E029E7150025019508750195
:100660008102950175088101050819012905950583
:10067000750191029501750391010507190029FF84
:10068000150025FF950675088100C00000000000D8
:10069000000000000000010204060A0F17202C3A97
:1006A0004A5D71879DB3C7DAE9F5FCFFFCF5E9DA2D
:1006B000C7B39D87715D4A3A2C20170F0A060402C2
:1006C00001000000000000000000000011241FBE17
:1006D000CFEFDAE0DEBFCDBF04B603FE27C08091C6
:1006E000ED019091EE01A091EF01B091F001873002
:1006F000904BA740B04BD1F41092ED011092EE0157
:100700001092EF011092F00114BE84B7877F84BF6E
:100710000FB6F894A895809160008861809360007E
:10072000109260000FBEE0E0FFE3099511E0A0E049
:10073000B1E0E8E9FAE402C005900D92A433B107F4
:10074000D9F721E0A4E3B1E001C01D92AD3EB207AC
:10075000E1F70E947C0B0C944A250C940000CF9387
:10076000DF93EC01623709F4B7C038F56A3609F453
:100770007DC098F4663609F461C048F4643609F423
:1007800051C008F055C0662309F441C006C168365F
:1007900009F460C008F458C063C06E3609F484C020
:1007A00030F46C3609F46EC008F466C077C0603768
:1007B00009F486C008F47EC089C06A3709F4BCC059
:1007C00080F4663709F4A0C030F4643709F490C0AF
:1007D00008F488C093C0683709F4A2C008F49AC02E
:1007E000A5C06E3709F4C0C030F46C3709F4B0C04E
:1007F00008F4A8C0B3C0603809F4C2C008F4BAC095
:10080000613809F4C3C0623809F442C0C6C08A81A5
:10081000882321F085EE0E94EA11BEC085EE0E9479
:10082000B212BAC00E94401A8A818111B9C0B5C003
:100830000E94401A8A818111B6C0AFC00E94401A3E
:100840008A818111B3C0A9C00E94401A8A81811196
:10085000B0C0A3C00E94401A8A818111ADC09DC062
:100860000E94401A8A818111AAC097C00E94401A32
:100870008A818111A7C091C00E94401A8A8181118A
:10088000A4C08BC00E94401A8A818111A1C085C07A
:100890000E94401A8A8181119EC07FC00E94401A26
:1008A0008A8181119BC079C00E94401A8A8181117E
:1008B00098C073C00E94401A8A81811195C06DC092
:1008C0000E94401A8A81811192C067C00E94401A1A
:1008D0008A8181118FC061C00E94401A8A81811172
:1008E0008CC05BC00E94401A8A81811189C055C0AA
:1008F0000E94401A8A81811186C04FC00E94401A0E
:100900008A81811183C049C00E94401A8A81811165
:1009100080C043C00E94401A8A8181117DC03DC0C1
:100920000E94401A8A8181117AC037C00E94401A01
:100930008A81811177C031C00E94401A8A81811159
:1009400074C02BC00E94401A8A81811171C025C0D9
:100950000E94401A8A8181116EC01FC00E94401AF5
:100960008A8181116BC019C00E94401A8A8181114D
:1009700068C013C00E94401A8A81811165C00DC0F1
:100980000E94401A8A81811162C007C00E94401AE9
:100990008A8181115FC001C060C020E030E05CC08E
:1009A00026E232E059C029E132E056C02CE032E0C4
:1009B00053C02FEF31E050C022EF31E04DC025EEA3
:1009C00031E04AC028ED31E047C02FEC31E044C0AF
:1009D00026EC31E041C029EB31E03EC020EB31E0B4
:1009E0003BC023EA31E038C02AE931E035C021E9D3
:1009F00031E032C024E831E02FC027E731E02CC0DD
:100A00002EE631E029C021E631E026C024E531E0C0
:100A100023C02BE431E020C02EE331E01DC025E3EC
:100A200031E01AC02CE231E017C023E231E014C0FB
:100A30002AE131E011C02DE031E00EC024E031E0C8
:100A40000BC02BEF30E008C022EF30E005C029EEEC
:100A500030E002C020EE30E0C901DF91CF9108956F
:100A600008956091B1017091B2018091B3019091AC
:100A7000B4010E943A1C56985E9825982D982698A5
:100A80002E9827982F98813019F0823021F0089500
:100A9000259A2D9A0895269A2E9A08950C94310538
:100AA00056985E9825982D9826982E9827982F98D6
:100AB0008FEF90E0909389008093880090938B0053
:100AC00080938A0090938D0080938C00259A2D9AB4
:100AD0002FEF80E792E0215080409040E1F700C086
:100AE0000000269A2E9A2FEF80E792E02150804056
:100AF0009040E1F700C00000279A2F9A2FEF80E77F
:100B000092E0215080409040E1F700C0000025981D
:100B10002D982FEF80E792E0215080409040E1F740
:100B200000C0000026982E982FEF80E792E0215019
:100B300080409040E1F700C0000027982F98569819
:100B40005E9825982D9826982E9827982F98089586
:100B500089EA8093800089E08093810024982C9812
:100B60003F988AB18F748AB96E98479A8BB1806B1F
:100B70008BB9769A0E9450050C94300580E28093E0
:100B800000018091340181110EC00E940D0681E0A8
:100B9000809334012FEF83ED90E32150804090400B
:100BA000E1F700C0000080E40E941306809300017A
:100BB00081112EC00E943D0680930001811128C042
:100BC0000E943D0680930001811122C08FE30E94A4
:100BD0003D068093000181111BC00E94350680E410
:100BE0000E94130680930001811112C08CE00E94C4
:100BF0003D068093000181110BC00E943D06809349
:100C00000001811105C08FE30E943D068093000121
:100C10000E9435068091000108951092B9008AE083
:100C20008093B800089594EA9093BC009091BC0022
:100C300097FFFCCF9091B900987F983021F09031C8
:100C400011F081E008958093BB0084E88093BC009C
:100C50008091BC0087FFFCCF8091B900887F8831EC
:100C600011F0803471F780E0089584E98093BC002E
:100C70008091BC0084FDFCCF08958093BB0084E884
:100C80008093BC008091BC0087FFFCCF9091B9009D
:100C9000987F81E0983209F480E0089584E8809399
:100CA000BC008091BC0087FFFCCF8091BB00089501
:100CB00080910001811115C080E40E941306809389
:100CC000000181110CC082E10E943D068093000169
:100CD000811105C08FEF0E943D06809300010E94A4
:100CE000350684B1807F84B985B1807F85B98AB1AA
:100CF000837F8AB98BB1837F8BB93E9846980895DC
:100D00000E94BE05809300010E94580680B38C703B
:100D100080BB81B3836F81BBE4E4F1E0A6E3B1E083
:100D200011921D9281E0E235F807D1F70C94A805E5
:100D30009F92AF92BF92CF92DF92EF92FF920F936A
:100D40001F93CF93DF9380910001882379F08091E6
:100D500035018F5F80933501811108C00E94BE0567
:100D600080930001811102C00E94500586E3E82EA5
:100D700081E0F82E8701C0E0D0E0BB24B39492E07C
:100D8000A92ECC24C394D12CC730D10500F5809175
:100D90000001811164C080E40E9413068093000169
:100DA000811112C082E10E943D06809300018111F1
:100DB0000BC0C6010C2E01C0880F0A94EAF780957B
:100DC0000E943D06809300010E94350648C0CA304B
:100DD000A1F028F4C83059F0C93061F005C0CC301A
:100DE00089F070F0CD3089F0209A289810C0219AAF
:100DF00029980DC0229A2A980AC0239A2B9807C0D6
:100E0000529A01C0539A5B9802C03E9A4698E0EA13
:100E1000EA95F1F78FB181708B25799902C032E0A4
:100E200001C030E0832B7C9902C034E001C030E087
:100E3000832B7D9902C028E001C020E0822B7E999F
:100E400002C090E101C090E0892B9FB19095991F5D
:100E50009927991F9295990F907E892B0FC08091A9
:100E6000000181114AC080E40E94130680930001B2
:100E7000882381F1912C0E943506892DD8019C91FF
:100E8000981719F08C93A09201010E9458062196A0
:100E90000F5F1F4FCE30D10509F076CF8091010151
:100EA000882369F1815080930101882339F0EFE9AB
:100EB000FFE03197F1F700C0000021C0E4E4F1E069
:100EC000D7018D917D018193B4E4EB16B1E0FB066F
:100ED000B9F715C083E10E943D068093000181119E
:100EE000C9CF81E40E941306809300018111C2CF13
:100EF0000E944E06982E9094BECF80E0BFCF0E94F5
:100F00004E0581E0DF91CF911F910F91FF90EF90FF
:100F1000DF90CF90BF90AF909F900895E82FF0E0C2
:100F2000EC5BFE4F8081089508958B3B910580F422
:100F3000883A910548F5853A9105D8F484309105B1
:100F400008F0B2C0019709F06EC081E090E008950A
:100F5000803E910508F467C0883E910508F4A4C05E
:100F60009C01205F31092031310508F05CC090659B
:100F70000895853A910509F459C0863A910509F01A
:100F800058C082E890E40895883A910509F454C065
:100F9000893A910509F453C08A3A910509F452C07F
:100FA0008B3A910509F451C08C3A910509F450C06F
:100FB0008D3A910509F44FC0803B910509F44EC06C
:100FC0008E3A910509F44DC08F3A910509F44CC051
:100FD000813B910509F44BC0823B910509F44AC05D
:100FE000833B910509F449C0843B910509F448C04D
:100FF000853B910509F447C0863B910509F446C03D
:10100000873B910509F445C0883B910509F444C02C
:10101000893B910509F443C08A3B910509F442C01C
:1010200080E094E4089580E090E0089581E890E401
:10103000089583E890E4089582EE94E4089589EE9B
:1010400094E408958AEE94E4089585EB94E4089579
:1010500086EB94E4089587EB94E408958CEC94E493
:1010600008958DEC94E4089583E895E408958AE862
:1010700095E4089582E995E4089584E995E4089556
:1010800081E296E4089583E296E4089584E296E48A
:10109000089585E296E4089586E296E4089587E24D
:1010A00096E408958AE296E40895089524E5829FDF
:1010B000C0011124FC0126E0729FE00DF11D1124F6
:1010C000E60FF11DEE0FFF1FE35CFD4F859194913C
:1010D0000895880F991FFC01ED54FF4F859194915D
:1010E0000895880F991FFC01ED5CFD4F8591949147
:1010F000089524E5829FC0011124FC0146E0749FFD
:10110000E00DF11D1124E60FF11DEE0FFF1FE35C52
:10111000FD4F859194919C013A9521154FE134073B
:1011200008F425C13F512115304120F49F700E94E1
:10113000710808959C0130532115304118F4992706
:10114000906C0895811520E5920769F40E942B1692
:101150004FEF84E39CE0415080409040E1F700C0B5
:1011600000000C94321D813020E5920731F480910B
:10117000CC0181608093CC0108959C0130552115EC
:10118000304108F05CC0292F33272F7033272130DE
:101190003105E9F4AC0164E0440F551F6A95E1F7AD
:1011A00044275370BC016370772702C0220F331F9E
:1011B0006A95E2F73C68242B352B73E0880F991F62
:1011C0007A95E1F780769927822B932B0895223028
:1011D000310529F4982F8827816F906A089523306C
:1011E0003105A1F4AC0133E0440F551F3A95E1F706
:1011F000407E57708370992721E030E002C0220FB3
:10120000331F8A95E2F7C9019C6816C02430310566
:1012100031F5AC0123E0440F551F2A95E1F7407EDC
:1012200057708370992721E030E002C0220F331FEE
:101230008A95E2F7C9019A68842B952B08959C0141
:1012400030572115304118F49F70906208959C0129
:1012500030582115304118F49F70906A0895803EEF
:101260009105E0F4803C910558F58133910509F42E
:101270006FC048F48932910509F463C08A32910540
:1012800009F46DC072C089339105E9F08238910587
:10129000D1F08533910509F44DC067C0833E9105B7
:1012A00081F138F4803E9105B9F0823E9105D9F084
:1012B0005CC0863E910561F1873E9105A1F155C064
:1012C0000E94690808952091DE0120FD02C021FFDF
:1012D0004CC080EE90E049C08091DE0180FFF9CFE4
:1012E00089E390E042C08091DE0182FF0EC08091D0
:1012F000DE0184FF03C080E090E037C083EE90E021
:1013000034C08091DE0182FFF2CF82EE90E02DC0EA
:101310008091DE0183FF0BC08091DE0184FDEBCF65
:1013200087EE90E022C08091DE0183FFF5CF86EE4C
:1013300090E01BC08091DE0185FF07C089E290E04C
:1013400014C08091DE0185FFF9CF85E390E00DC0E8
:101350008091DE0186FF07C08AE290E006C080919E
:10136000DE0186FFF9CF81E390E00E9495070895A2
:101370000895809162010895CF93DF9300D01F926A
:10138000CDB7DEB79C018091E401843019F593E07C
:1013900099833B832A839093E9008FEF9091E80033
:1013A000815095FD06C095ED9A95F1F700008111E9
:1013B000F5CF8091E80085FF0DC040E050E063E08C
:1013C00070E0CE0101960E94290C8091E8008E7792
:1013D0008093E8000F900F900F90DF91CF910895C8
:1013E000CF93DF9300D01F92CDB7DEB72091E401F9
:1013F000243021F522E029839B838A8383E0809334
:10140000E9008FEF9091E800815095FD06C095EDC1
:101410009A95F1F700008111F5CF8091E80085FFE2
:101420000DC040E050E063E070E0CE0101960E9404
:10143000290C8091E8008E778093E8000F900F9040
:101440000F90DF91CF9108959C018091E401843049
:10145000F9F482E08093E9009FEF8091E8009150D9
:1014600085FD06C085ED8A95F1F700009111F5CF55
:101470008091E80085FF0CC040E050E065E070E03E
:10148000C9010E94290C8091E8008E778093E800C2
:101490000895CF93DF93EC018091E401843009F04B
:1014A00046C090910C019923D9F090910D01992398
:1014B000B9F08093E9008FEF9091E800815095FD9D
:1014C00006C095E19A95F1F700008111F5CF809162
:1014D000E80085FF2CC040E050E060E170E017C0FC
:1014E00081E08093E9008FEF9091E800815095FDB5
:1014F00006C095ED9A95F1F700008111F5CF809126
:10150000E80085FF14C040E050E068E070E0CE01E4
:101510000E94290C8091E8008E778093E80080E19A
:10152000FE01A2E5B1E001900D928A95E1F7DF910D
:10153000CF9108958091E301811109C00E94BA0DF5
:101540000E94170E8091E20084608093E20008956B
:101550001092E301089508950C9468230E94C81C1A
:101560000E946E230E94C2100C94B80942E061EC04
:1015700081E00E94330D42E061EC82E00E94330D75
:1015800042E061EC83E00E94330D42E161EC84E0D3
:101590000C94330D8091E601833009F455C030F48A
:1015A000813071F0823009F48EC008958A3009F4D8
:1015B0007AC08B3009F460C0893009F09CC020C02B
:1015C0008091E501813A09F096C08091E800877F1B
:1015D0008093E8008091E9019091EA01892B21F440
:1015E00060E182E591E003C060E080E090E070E0BF
:1015F0000E94740C8091E8008B778093E800089536
:101600008091E501813209F076C08091E9019091E5
:10161000EA01009719F0039709F06DC08091E80086
:10162000877F8093E8008091E80082FD05C080916B
:10163000E4018111F8CF5FC08091F10080936201D5
:101640008091E8008B7753C08091E501813A09F0E1
:1016500052C08091E9019091EA01892B09F04BC0B9
:101660008091E800877F8093E8008091E80080FF08
:10167000FCCF80910C0136C08091E5018132D9F513
:101680008091E9019091EA01892BA9F58091E80008
:10169000877F8093E8000E94680D8091E701809326
:1016A0000C010C942B168091E501813221F580917B
:1016B000E800877F8093E8000E94680D8091E80130
:1016C0008093630108958091E501813AA1F48091AE
:1016D000E800877F8093E8008091E80080FFFCCFDE
:1016E000809163018093F1008091E8008E77809370
:1016F000E8000C94680D089584B7877F84BF0FB607
:10170000F894A895809160008861809360001092A1
:1017100060000FBE90E080E80FB6F89480936100FF
:10172000909361000FBE0E9411110E94BA0D0E9499
:10173000170E8091E20084608093E20078940E940A
:10174000A2100E94131182E091E00E94BD100E943D
:1017500056238091E401853069F40E948A1C8091AF
:10176000E2018823B1F30E94B41C882391F30E9404
:10177000130CEFCF0E941911ECCF292F3327233000
:101780003105C9F060F42130310581F02230310596
:1017900009F041C08DE690E021E135E040C0213202
:1017A0003105E1F02232310531F135C082E190E0BE
:1017B0002EE735E034C099278130910549F028F0B3
:1017C000029749F5EDEDF4E005C0EDE0F5E002C06B
:1017D000E5EFF4E0849190E09F0121C06430D8F4FB
:1017E000E62FF0E0EE0FFF1FEE5DFE4F208131810E
:1017F00089E090E014C0643070F470E0FB01EE0FFB
:10180000FF1FE65EFE4F20813181FB01EA5EFE4F45
:10181000808190E004C080E090E020E030E0FA01B8
:1018200031832083089580E189BD82E189BD09B4B7
:1018300000FEFDCF8091D8008F7D8093D8008091ED
:10184000E00082608093E0008091E00081FDFCCFA9
:101850000895CF92DF92EF92FF920F931F93CF9351
:10186000DF93EC018B016A010E94870D811133C067
:10187000C114D10439F0F60180819181081B190B44
:10188000C80FD91FE12CF12C0115110519F1809118
:10189000E80085FD16C08091E8008E778093E8000F
:1018A000C114D10449F0F60180819181E80EF91E3E
:1018B000F182E08285E00FC00E94870D882321F32A
:1018C0000AC089918093F10001501109FFEFEF1ACE
:1018D000FF0ADACF80E0DF91CF911F910F91FF9047
:1018E000EF90DF90CF9008952091EB013091EC01C3
:1018F0002617370748F06115710539F42091E80083
:101900002E772093E80001C0B901FC0120E06115A9
:10191000710579F18091E4018823F1F18530F1F1CD
:101920008091E80083FD3CC08091E80082FD2EC0DC
:101930008091E80080FFEBCF2091F3008091F200CE
:1019400090E0922B6115710551F08830910538F4C3
:1019500021912093F100615071090196F3CF21E0AC
:10196000089709F020E08091E8008E778093E800E6
:10197000CECF2111CFCF0AC08091E401882361F03E
:10198000853061F08091E80083FD0AC08091E80015
:1019900082FFF2CF80E0089582E0089583E0089509
:1019A00081E008952091EB013091EC012617370773
:1019B00048F06115710539F42091E8002E772093E5
:1019C000E80001C0B901FC0120E06115710591F149
:1019D0008091E401882309F440C0853009F43FC0B8
:1019E0008091E80083FD3DC08091E80082FD2FC01A
:1019F0008091E80080FFE9CF2091F3008091F20010
:101A000090E0922B6115710559F08830910540F4F2
:101A100024912093F1003196615071090196F2CF23
:101A200021E0089709F020E08091E8008E7780930C
:101A3000E800CBCF2111CCCF0AC08091E4018823EC
:101A400061F0853061F08091E80083FD0AC08091EB
:101A5000E80082FFF2CF80E0089582E0089583E0FD
:101A6000089581E00895982F973068F59093E900E4
:101A7000981739F07091EC002091ED005091F00032
:101A800003C0242F762F50E021FD02C09F5FECCFD2
:101A90003091EB003E7F3093EB003091ED003D7FC5
:101AA0003093ED003091EB0031603093EB00709398
:101AB000EC002093ED005093F0002091EE0027FD04
:101AC000E5CF80E008958F708093E90081E008956C
:101AD0008091E50187FF11C08091E80082FD05C07B
:101AE0008091E4018111F8CF11C08091E8008B77DB
:101AF0000BC08091E401882349F08091E80080FFC9
:101B0000F8CF8091E8008E778093E80008952091C7
:101B1000E4003091E50095E64091EC00842F81705F
:101B200040FF23C08091E80080FD1DC08091E4014A
:101B3000882399F0853099F08091EB0085FD11C0E4
:101B40004091E4005091E5002417350729F39150A6
:101B500011F09A01E1CF84E0089582E0089583E0D6
:101B6000089581E0089580E008954091E80042FFE3
:101B7000DDCF08950E94280E0E94300EE0EEF0E0C6
:101B8000808181608083E8EDF0E080818F778083C1
:101B900019BCA7EDB0E08C918E7F8C9380818F7EF5
:101BA00080831092E30108950F931F93CF93DF93E7
:101BB0000E94280E0E94300EC8EDD0E088818F77F9
:101BC000888388818068888388818F7D888319BC19
:101BD0001092E4011092E0011092E2011092E101F2
:101BE00000EE10E0F80180818B7F80838881816026
:101BF000888342E060E080E00E94330DE1EEF0E097
:101C000080818E7F8083E2EEF0E08081816080833E
:101C1000808188608083F80180818E7F80838881C5
:101C200080618883DF91CF911F910F910895E8ED36
:101C3000F0E080818F7E8083E7EDF0E0808181603D
:101C4000808384E082BF81E08093E3010C94D40D13
:101C5000E8EDF0E080818E7F80831092E2000895AD
:101C60001092DA001092E10008951F920F920FB6C1
:101C70000F9211242F933F934F935F936F937F9312
:101C80008F939F93AF93BF93EF93FF938091E10066
:101C900082FF0BC08091E20082FF07C08091E100CB
:101CA0008B7F8093E1000E94A1108091DA0080FF79
:101CB0001FC08091D80080FF1BC08091DA008E7F0A
:101CC0008093DA008091D90080FF0DC080E189BD4A
:101CD00082E189BD09B400FEFDCF81E08093E4017B
:101CE0000E949A0A05C019BC1092E4010E94A80A39
:101CF0008091E10080FF19C08091E20080FF15C053
:101D00008091E2008E7F8093E2008091E20080610A
:101D10008093E2008091D80080628093D80019BC43
:101D200085E08093E4010E94AC0A8091E10084FF89
:101D300030C08091E20084FF2CC080E189BD82E147
:101D400089BD09B400FEFDCF8091D8008F7D8093BE
:101D5000D8008091E1008F7E8093E1008091E200C5
:101D60008F7E8093E2008091E20081608093E200A8
:101D70008091E001882311F084E007C08091E300A6
:101D800087FD02C081E001C083E08093E4010E94EE
:101D9000AE0A8091E10083FF29C08091E20083FFB9
:101DA00025C08091E100877F8093E10082E08093ED
:101DB000E4011092E0018091E1008E7F8093E100C8
:101DC0008091E2008E7F8093E2008091E20080614A
:101DD0008093E20042E060E080E00E94330D809159
:101DE000F00088608093F0000E94AB0AFF91EF91B1
:101DF000BF91AF919F918F917F916F915F914F9123
:101E00003F912F910F900FBE0F901F9018951F922A
:101E10000F920FB60F9211242F933F934F935F931E
:101E20006F937F938F939F93AF93BF93CF93DF93E2
:101E3000EF93FF93C091E900CF708091EC00D82F11
:101E4000D17080FDD0E81092E9008091F000877F8A
:101E50008093F00078940E944B0F1092E9008091DB
:101E6000F00088608093F000CD2BCF70C093E90024
:101E7000FF91EF91DF91CF91BF91AF919F918F91A2
:101E80007F916F915F914F913F912F910F900FBE76
:101E90000F901F9018951F93CF93DF93CDB7DEB7A8
:101EA000AA970FB6F894DEBF0FBECDBFE5EEF1E006
:101EB0008091F100819321E0ED3EF207C9F70E9485
:101EC000CA0A8091E80083FF24C18091E5019091C6
:101ED000E601492F50E04A30510508F01AC1FA01D5
:101EE000EA5AFF4F0C94FF24803881F0823809F0C1
:101EF00010C18091E9018F708093E9008091EB001F
:101F000085FB882780F91092E90006C08091E101E5
:101F10009091E201911182609091E800977F9093F7
:101F2000E8008093F1001092F100C8C0282F2D7FA7
:101F300009F0EFC0882319F0823061F0EAC0809187
:101F4000E701813009F0E5C0933009F080E080932B
:101F5000E2012BC08091E701811127C08091E90146
:101F60008F7009F4D6C08093E9002091EB0020FF28
:101F70001CC0933021F48091EB00806214C09091DA
:101F8000EB0090619093EB0021E030E0A90102C0EA
:101F9000440F551F8A95E2F74093EA001092EA0039
:101FA0008091EB0088608093EB001092E9008091B3
:101FB000E800877F86C08111ACC01091E7011F77D0
:101FC0008091E3008078812B8093E3008091E8008A
:101FD000877F8093E8000E94680D8091E80080FF71
:101FE000FCCF8091E30080688093E300111102C070
:101FF00082E001C083E08093E4018BC0805882308E
:1020000008F087C08091E7019091E8018C3D53E092
:10201000950779F583E08A838AE289834FB7F8943C
:10202000DE01139620E03EE051E2E32FF0E0509312
:102030005700E49120FF03C0E295EF703F5FEF701F
:102040008E2F90E0EA3010F0C79601C0C0968D93B5
:102050009D932F5F243149F74FBF8091E800877F20
:102060008093E8006AE270E0CE0101960E94740C51
:1020700014C0AE014F5F5F4F6091E9010E94BD0B3C
:10208000BC01892B09F445C09091E800977F90939B
:10209000E80089819A810E94D20C8091E8008B77B8
:1020A0008093E80036C08038A1F58091E800877FF2
:1020B0008093E8008091E0018093F1008091E80036
:1020C0008E778093E8000E94680D23C0811121C0A3
:1020D0008091E7019091E80199270297D4F48091CB
:1020E000E800877F8093E8008091E7018093E0011A
:1020F0000E94680D8091E001811106C08091E3008B
:1021000087FD02C081E001C084E08093E4010E9469
:10211000B60A8091E80083FF0AC08091E800877FBB
:102120008093E8008091EB0080628093EB00AA9698
:102130000FB6F894DEBF0FBECDBFDF91CF911F91D8
:1021400008950895CF938091E4018823A1F0C09170
:10215000E900CF709091EC00892F817090FD80E8AC
:10216000C82B1092E9008091E80083FD0E944B0F7C
:10217000CF70C093E900CF91089590936901809347
:1021800068010895E0916801F0916901309721F0AC
:102190000190F081E02D099480E00895E0916801BC
:1021A000F0916901309721F00280F381E02D0994CC
:1021B0000895E0916801F0916901309721F0048061
:1021C000F581E02D09940895209166013091670111
:1021D0002817390771F09093670180936601E091A9
:1021E0006801F0916901309721F00680F781E02DB8
:1021F00009940895209164013091650128173907E9
:1022000071F09093650180936401E0916801F09111
:102210006901309721F00084F185E02D099408953B
:1022200008950C9410110E94CE1C0E9480060C94FC
:10223000941DCF92DF92EF92FF920F931F93CF9353
:10224000DF93CDB7DEB72B970FB6F894DEBF0FBE86
:10225000CDBF0E9498068BE6C82E81E0D82E00E004
:1022600010E0E02E802F0E948E07F60141916F0151
:10227000F82EF426B1F40F5F1F4F0E30110589F7C9
:102280008FEF89838A831B820E94D71C8160782FFD
:102290009D838C8349815A816B818D810E94BC1101
:1022A00040C09091CC0191FF04C08B870E9494079D
:1022B0008B8520E030E04F2D50E0922FBA01022EA6
:1022C00002C0759567950A94E2F760FF24C02E83DB
:1022D000EF8221E030E0690102C0CC0CDD1C9A9550
:1022E000E2F790E08C219D21892B09F420E02887DA
:1022F0000E94D71C8160782F9A8789874E815F81E1
:1023000068858A850E94BC11F801E559FE4F8081DD
:10231000C826C08206C02F5F3F4F2630310569F6C0
:10232000AACF0E947B200E94C21090916A01891757
:10233000A1F00E94C21080936A012B960FB6F89408
:10234000DEBF0FBECDBFDF91CF911F910F91FF90E8
:10235000EF90DF90CF900C94B8092B960FB6F894BD
:10236000DEBF0FBECDBFDF91CF911F910F91FF90C8
:10237000EF90DF90CF900895CF93DF93CDB7DEB786
:102380002B970FB6F894DEBF0FBECDBF4F83588793
:1023900069877A878B87DE01119686E0FD011192AD
:1023A0008A95E9F785E0FE01379601900D928A95AE
:1023B000E1F749815A816B817C818D819E810E94E8
:1023C000BF182B960FB6F894DEBF0FBECDBFDF91BE
:1023D000CF910895CF93C82F882309F4C1C08238C4
:1023E00059F40E94C21081FDBBC089E30E945C1BAE
:1023F0000E94141C89E30CC0833879F40E94C21037
:1024000080FDAEC083E50E945C1B0E94141C83E526
:102410000E949B1BCF910C94141C843859F40E9489
:10242000C21082FD9DC087E40E945C1B0E94141CA8
:1024300087E4EECF8CEF8C0F813A48F48C2F0E940A
:10244000BB2281118DC08C2F0E945C1BE3CF80E2E8
:102450008C0F883048F4C77081E001C0880FCA959E
:10246000EAF70E94DD1BD6CF8BE58C0F833078F422
:10247000C53A29F0C63A31F083E890E005C081E81A
:1024800090E002C082E890E0CF910C94E41088E5DF
:102490008C0F833108F064C0C83A39F1C93A41F170
:1024A000CA3A49F1CB3A51F1CC3A59F1CD3A61F1FE
:1024B000C03B69F1CE3A71F1CF3A79F1C13B81F17C
:1024C000C23B89F1C33B91F1C43B99F1C53BA1F1FA
:1024D000C63BA9F1C73BB1F1C83BB9F1C93BC1F15A
:1024E000CA3BC9F180E090E038C082EE90E035C090
:1024F00089EE90E032C08AEE90E02FC085EB90E04C
:102500002CC086EB90E029C087EB90E026C08CECD5
:1025100090E023C08DEC90E020C083E891E01DC0E6
:102520008AE891E01AC082E991E017C084E991E05D
:1025300014C081E292E011C083E292E00EC084E216
:1025400092E00BC085E292E008C086E292E005C00E
:1025500087E292E002C08AE292E0CF910C94FA10F6
:10256000CF910895882309F44BC0823859F40E9412
:10257000C21081FF45C089E30E945C1B0E94141CAD
:1025800089E30CC0833871F40E94C21080FF38C008
:1025900083E50E945C1B0E94141C83E50E949B1B28
:1025A0000C94141C843859F40E94C21082FF28C075
:1025B00087E40E945C1B0E94141C87E4EFCF9CEF11
:1025C000980F913A58F390E2980F983050F4877032
:1025D00091E001C0990F8A95EAF7892F0E94E31BC9
:1025E000DFCF9BE5980F933020F480E090E00C94CF
:1025F000E410885A833120F480E090E00C94FA10C3
:102600000895882321F00E94DD1B0C94141C08956A
:10261000882321F00E94E31B0C94141C0895BF92A0
:10262000CF92DF92EF92FF920F931F93CF93DF939E
:1026300000D000D000D0CDB7DEB77C0185E0F70137
:10264000DE01119601900D928A95E1F7F7018381E1
:102650009481892B09F4DDC2908181818F3F19F427
:102660009F3F09F4D6C2F7010281258122952F7080
:1026700099838A8389819A812E830E941B1B182F3C
:10268000B92E0E941A1B0E94E119EB2DE295EF7002
:102690004E2F50E0FA01E05AFF4F2E810C94FF2498
:1026A0008B2D807F9B2D9F70F92E882319F0F2943B
:1026B00080EFF822002349F0FF2009F457C28F2D44
:1026C0000E94ED1B0E94141C51C2812F0E94B21265
:1026D000FF2009F49EC28F2D0E94F31B26960FB691
:1026E000F894DEBF0FBECDBFDF91CF911F910F9148
:1026F000FF90EF90DF90CF90BF900C94141C3B2D77
:10270000307F8B2D8F70303211F08295807F1123B6
:1027100019F0113021F12CC00023B9F0222309F463
:1027200090C1213009F08DC126960FB6F894DEBF16
:102730000FBECDBFDF91CF911F910F91FF90EF9012
:10274000DF90CF90BF900C94FD1B222319F0213015
:1027500009F45FC28E830E94001C8E8186C1002313
:1027600021F0223008F055C26CC1211152C27DC146
:10277000002321F0222309F464C1F8C1222309F4C3
:1027800074C109C28B2D86958695837019F08130AE
:10279000D1F03FC2002321F0812F9B2D937002C006
:1027A00080E090E026960FB6F894DEBF0FBECDBF56
:1027B000DF91CF911F910F91FF90EF90DF90CF901D
:1027C000BF900C94E410002321F0812F9B2D937077
:1027D00002C080E090E026960FB6F894DEBF0FBEF0
:1027E000CDBFDF91CF911F910F91FF90EF90DF90C0
:1027F000CF90BF900C94FA10812F002319F00E9403
:10280000831F02C00E94EB1F26960FB6F894DEBF0E
:102810000FBECDBFDF91CF911F910F91FF90EF9031
:10282000DF90CF90BF900C9470208B2D837009F0B7
:1028300075C00111EEC1812F829586958770880F32
:10284000880F912F9F70C92ED12CE12CF12C082ECE
:1028500004C0CC0CDD1CEE1CFF1C0A94D2F714FF44
:1028600012C00FE010E020E030E004C0000F111FA4
:10287000221F331F8A95D2F7C901B8016095709560
:102880008095909503C060E070E0CB014B2D46959C
:10289000469543704230C1F060F56C297D298E2940
:1028A0009F29413051F126960FB6F894DEBF0FBE36
:1028B000CDBFDF91CF911F910F91FF90EF90DF90EF
:1028C000CF90BF900C94081A6C297D298E299F29DE
:1028D00026960FB6F894DEBF0FBECDBFDF91CF9125
:1028E0001F910F91FF90EF90DF90CF90BF900C94CD
:1028F000241A0E94081AC701B60126960FB6F8944A
:10290000DEBF0FBECDBFDF91CF911F910F91FF9022
:10291000EF90DF90CF90BF900C94EC19002319F04A
:102920008B2D817001C08695882309F472C1812F97
:10293000829586958770880F880F912F9F70C92E7A
:10294000D12CE12CF12C082E04C0CC0CDD1CEE1C8B
:10295000FF1C0A94D2F714FF12C00FE010E020E031
:1029600030E004C0000F111F221F331F8A95D2F7D9
:10297000C901B801609570958095909503C060E09D
:1029800070E0CB014B2D4695469543704230C1F027
:1029900060F56C297D298E299F29413051F12696B9
:1029A0000FB6F894DEBF0FBECDBFDF91CF911F9160
:1029B0000F91FF90EF90DF90CF90BF900C94E21AB0
:1029C0006C297D298E299F2926960FB6F894DEBFA3
:1029D0000FBECDBFDF91CF911F910F91FF90EF9070
:1029E000DF90CF90BF900C94FE1A0E94E21AC701AC
:1029F000B60126960FB6F894DEBF0FBECDBFDF91AD
:102A0000CF911F910F91FF90EF90DF90CF90BF90EB
:102A10000C94C61A103FD1F118F4103E50F4A1C026
:102A2000123F09F463C008F44CC0133F09F473C0AB
:102A300098C01F708B2D8F710023A1F00E945F1A28
:102A4000812F26960FB6F894DEBF0FBECDBFDF9163
:102A5000CF911F910F91FF90EF90DF90CF90BF909B
:102A60000C9401130E94801A812F26960FB6F894B9
:102A7000DEBF0FBECDBFDF91CF911F910F91FF90B1
:102A8000EF90DF90CF90BF900C9408130023A9F033
:102A90002111BFC08B2D8F7126960FB6F894DEBF23
:102AA0000FBECDBFDF91CF911F910F91FF90EF909F
:102AB000DF90CF90BF900C94A51A223008F0A9C0E7
:102AC000E9CF0023A9F08B2D8F7126960FB6F894CD
:102AD000DEBF0FBECDBFDF91CF911F910F91FF9051
:102AE000EF90DF90CF90BF900C945F1A002359F3C2
:102AF0008B2D8F7126960FB6F894DEBF0FBECDBF1B
:102B0000DF91CF911F910F91FF90EF90DF90CF90C9
:102B1000BF900C94801A002399F08B2D8F7126960C
:102B20000FB6F894DEBF0FBECDBFDF91CF911F91DE
:102B30000F91FF90EF90DF90CF90BF900C944A1AC6
:102B400026960FB6F894DEBF0FBECDBFDF91CF91B2
:102B50001F910F91FF90EF90DF90CF90BF900C945A
:102B6000401A0023A9F0222309F4ADCF812F269625
:102B70000FB6F894DEBF0FBECDBFDF91CF911F918E
:102B80000F91FF90EF90DF90CF90BF900C94EA11DF
:102B9000222309F4ADCF812F26960FB6F894DEBF1D
:102BA0000FBECDBFDF91CF911F910F91FF90EF909E
:102BB000DF90CF90BF900C94B2124B2D4F70612FCD
:102BC000C7010E94AF0326960FB6F894DEBF0FBE72
:102BD000CDBFDF91CF911F910F91FF90EF90DF90CC
:102BE000CF90BF900C9464194B2D4F70612FC7018B
:102BF00026960FB6F894DEBF0FBECDBFDF91CF9102
:102C00001F910F91FF90EF90DF90CF90BF900C94A9
:102C1000550826960FB6F894DEBF0FBECDBFDF91E4
:102C2000CF911F910F91FF90EF90DF90CF90BF90C9
:102C300008950E94FA1B0E94CF1B0E94141C0E9440
:102C400020210E94702080E090E00E94E41080E04B
:102C500090E00C94FA100E94EA1B0C9419160E9442
:102C60001B1B292F22952F702C3030F42A3048F46A
:102C70002250223078F405C02C3041F02F3031F052
:102C800009C0803E48F0803F29F406C093FB8827A6
:102C900080F9089580E0089581E00895CF93DF934F
:102CA00000D000D01F92CDB7DEB70F900F900F90DD
:102CB0000F900F90DF91CF910895CF93DF9300D0C5
:102CC00000D000D0CDB7DEB726960FB6F894DEBFA1
:102CD0000FBECDBFDF91CF9108951F93CF93DF93A8
:102CE000C091790116E080917A01C81799F0D0E07F
:102CF0001C9FF0011D9FF00D1124E558FE4F4081EF
:102D0000518162817381848195810E945D16219633
:102D1000C770E9CFDF91CF911F9108954091AB012A
:102D20005091AC016091AD017091AE018091AF0105
:102D30009091B0010C945D168091B00182958F70D6
:102D400009F054C08091AD01882309F44FC08091EF
:102D50007901A0917A014091AE015091AF0160914B
:102D6000AB017091AC01B6E08A1709F43FC090E066
:102D700041155105C1F17F3F11F46F3FA1F1B89F9B
:102D8000F001B99FF00D1124E558FE4F2181271362
:102D90002AC02081261327C02281211124C023812B
:102DA00034812417350710F421503109241B350BC9
:102DB000283C3105C0F42091B0012F702061209390
:102DC000B00126E0289FF001299FF00D1124E05862
:102DD000FE4F80818F70806180838BEA91E00E943A
:102DE0000F130C946D1601968770BECF0895CF9285
:102DF000DF92EF92FF920F931F93CF93DF93CDB7A4
:102E0000DEB762970FB6F894DEBF0FBECDBF8C0160
:102E100085E0F801DE011D9601900D928A95E1F79B
:102E2000D8014C9111965C91119712966C918091FA
:102E3000AE019091AF01009709F475C13091AB01DB
:102E40007091AC017F3F19F43F3F09F46CC1F80168
:102E5000C380D480E090AD01EE2009F4BEC0209183
:102E6000B001C816D90628F0D601A81BB90BCD01B0
:102E700004C0809590958C0D9D1DFF24F394883C93
:102E8000910578F0F12C207F09F0C4C07C2DD98AFF
:102E9000C88A89890E944E168BEA91E00E940F131E
:102EA000AFC0822F807F09F045C0571313C0431372
:102EB00011C061110FC02F7020612093B0010E94DA
:102EC0008E168BEA91E00E940F138091B001F801F9
:102ED00085832EC0CD2819F15F3F11F44F3FF9F0E3
:102EE000F62E61111CC08091790120917A0136E0A3
:102EF000821709F45BC090E0389FF001399FF00D14
:102F00001124E558FE4F7181571306C07081471395
:102F100003C07281711103C001968770E9CFF62E4C
:102F2000662309F41CC18091B00181608093B001D7
:102F3000F12C15C1571309C0431307C0611105C017
:102F40008091B001F8018583C8C04D875E878D856B
:102F50009E856A8B0E942F166A898823D1F1662389
:102F6000C1F12091B001822F82958F7090E002977D
:102F700074F08091AB019091AC0198878F83198692
:102F8000DB86CA862C87CE0107960E940F1386E047
:102F9000F801ABEAB1E001900D928A95E1F70E9449
:102FA0009C160E948E16FF24F394D9C04D875E872D
:102FB0008D859E850E941B1B292F22952F70223004
:102FC00008F0C1C09F7009F0BBC0805E883008F473
:102FD000C6C0C8010E940F13E6CFC816D90608F470
:102FE00053C0F601E81BF90BCF01883C910508F4AA
:102FF00050C0F12C7C2DD98AC88A89890E944E162E
:10300000EBEAF1E086E0DF011D928A95E9F70E9484
:103010008E16A5C0571314C0431312C0611110C0FF
:103020008091B001F8018583C8010E940F1386E0EA
:10303000EBEAF1E0DF011D928A95E9F7FE2C8FC0E3
:103040004D875E878D859E856A8B0E942F166A89C3
:10305000882309F4BECF662309F4BBCF2091B001C9
:10306000822F82958F7090E002970CF490CF809120
:10307000AB019091AC019A8389831B82DD82CC8263
:103080002E83CE01019681CF809590958C0D9D1D4C
:10309000ACCFF62E662309F49CCF571333C04313ED
:1030A00031C02091B00120FD24C0822F82958F7005
:1030B000482F50E041155105E1F0D80115962C93A9
:1030C00015974F30510549F08F5F982F9295907F5B
:1030D000822F8F70892B15968C93C8010E940F1335
:1030E00086E0F801ABEAB1E001900D928A95E1F734
:1030F0008ECF86E0F801ABEAB1E001900D928A959F
:10310000E1F72DC04D875E878D859E850E942F1625
:1031100081113DCF8091B00181608093B001C801E1
:103120000E940F131CC0662309F453CF4D875E879E
:103130008D859E850E942F16882309F44ACF27CFBC
:10314000811143CF0CC0243008F043CF9F7009F4A5
:103150003CCFD80115969C91907F09F036CF8F2DEA
:1031600062960FB6F894DEBF0FBECDBFDF91CF9150
:103170001F910F91FF90EF90DF90CF9008951F93D4
:10318000CF93DF93CDB7DEB72C970FB6F894DEBFA1
:103190000FBECDBF4F83588769877A878B879C87FF
:1031A000CE0107960E94F716882371F08A859B85C9
:1031B000892B09F441C088858F3F09F065C08F8154
:1031C0008F3F09F061C038C086E0FE013796DE010E
:1031D000119601900D928A95E1F76A857B856115BC
:1031E000710551F1FF81E885EF3F11F4FF3F21F1B7
:1031F00020917A0130E0C9010196877099274091AA
:10320000790150E08417950709F447C0F983EA83F0
:103210007D836C8396E0929FD001939FB00D112423
:10322000A558BE4FFE01319601900D929A95E1F797
:1032300080937A010E946D1616E080917901909139
:103240007A018917B9F1189FC001112485589E4F42
:103250000E94F716882371F1E09179011E9FF00119
:103260001124E558FE4F4081518162817381848130
:1032700095810E945D168091790190E0019687709A
:10328000992780937901D9CF4F81588569857A85AF
:103290008B859C850E945D16CFCF0E942B161092C5
:1032A0007A0110927901EBEAF1E086E0DF011D92EC
:1032B0008A95E9F72C960FB6F894DEBF0FBECDBF06
:1032C000DF91CF911F910895EF92FF920F931F937B
:1032D000CF93DF938C01892B09F46CC0F12CEE2481
:1032E000E394E8012196F8018491843740F4843016
:1032F00008F051C0813081F0823019F15BC0853710
:1033000009F444C0A8F19CE7980F903708F052C028
:103310008F770E94B21241C00E5F1F4FFE01849151
:1033200090E2980F983050F48770FE2D01C0FF0F87
:103330008A95EAF78F2F0E94ED1B14C00E94EA11B4
:103340002DC00E5F1F4FFE01849190E2980F9830C0
:1033500060F48770FE2D01C0FF0F8A95EAF78F2F6A
:103360000E94F31B0E94141C19C00E94B21216C0C6
:103370000E5F1F4FFE01C491CC2381F08FE99FE0C7
:103380000197F1F700C00000C150F6CF0E5F1F4F4C
:10339000FE01F49003C00E94EA118E018F2D882354
:1033A00009F49FCFEFE9FFE03197F1F700C000008B
:1033B0008150F5CFDF91CF911F910F91FF90EF904A
:1033C000089508956093B5017093B6018093B70195
:1033D0009093B8010C9419160F931F930091B501A7
:1033E0001091B6012091B7013091B801DC01CB01F9
:1033F000802B912BA22BB32B8093B5019093B60118
:10340000A093B701B093B8011F910F910C941916B6
:103410000F931F930091B5011091B6012091B70150
:103420003091B801DC01CB0180239123A223B32387
:103430008093B5019093B601A093B701B093B80102
:103440001F910F910C9419160F931F930091B501C2
:103450001091B6012091B7013091B801DC01CB0188
:1034600080279127A227B3278093B5019093B601B7
:10347000A093B701B093B8011F910F910C94191646
:103480001092B1011092B2011092B3011092B401E6
:103490000C94191641E050E060E070E004C0440F65
:1034A000551F661F771F8A95D2F74093B10150933D
:1034B000B2016093B3017093B4010C94191641E00A
:1034C00050E060E070E004C0440F551F661F771F96
:1034D0008A95D2F78091B1019091B201A091B30188
:1034E000B091B401482B592B6A2B7B2B4093B1012F
:1034F0005093B2016093B3017093B4010C94191608
:1035000041E050E060E070E004C0440F551F661FCA
:10351000771F8A95D2F74095509560957095809168
:10352000B1019091B201A091B301B091B4014823CF
:1035300059236A237B234093B1015093B2016093D6
:10354000B3017093B4010C94191641E050E060E0AF
:1035500070E004C0440F551F661F771F8A95D2F78D
:103560008091B1019091B201A091B301B091B401E9
:10357000482759276A277B274093B1015093B2010E
:103580006093B3017093B4010C9419160F931F93B9
:103590000091B1011091B2012091B3013091B401B9
:1035A000DC01CB01802B912BA22BB32B8093B1019B
:1035B0009093B201A093B301B093B4011F910F9106
:1035C0000C9419160F931F930091B1011091B20141
:1035D0002091B3013091B401DC01CB018023912310
:1035E000A223B3238093B1019093B201A093B301BE
:1035F000B093B4011F910F910C9419160F931F9360
:103600000091B1011091B2012091B3013091B40148
:10361000DC01CB0180279127A227B3278093B1013A
:103620009093B201A093B301B093B4011F910F9195
:103630000C9419160895CF92DF92EF92FF920F9398
:103640001F93CF93DF938C01C090B101D090B20152
:10365000E090B301F090B4018091B5019091B60172
:10366000A091B701B091B801C82AD92AEA2AFB2A49
:10367000CFE1D0E0D701C6010C2E04C0B695A795C6
:10368000979587950A94D2F780FF07C0B8018C2FD1
:103690000E9479088130910531F4219758F7B801DB
:1036A00080E00E947908DF91CF911F910F91FF90E8
:1036B000EF90DF90CF90089590910C019923F1F055
:1036C00090910D019923D1F0982F96959695969506
:1036D0009F3080F5E0910E01F0910F01E90FF11D8F
:1036E000877021E030E0A90102C0440F551F8A9580
:1036F000E2F7CA019181892B8183089520910E01FF
:1037000030910F01F90132969FEF40E051918517FA
:1037100089F09F3F19F4511101C0942F4F5F4E3033
:10372000A9F79F3F39F0F901E90FF11D97FDFA95CF
:1037300082830895089590910C019923F9F0909156
:103740000D019923D9F0982F9695969596959F30CF
:1037500028F5E0910E01F0910F01E90FF11D87703E
:1037600021E030E0A90102C0440F551F8A95E2F71D
:10377000CA018095918189238183089520910E014A
:1037800030910F01F9013296205F3F4F90818913EC
:1037900001C010823196E217F307C1F7089581E066
:1037A00090E0E0910E01F0910F01E80FF91F1082F7
:1037B000019680319105A9F708959091CB01892B4D
:1037C0008093CB01089580959091CB0189238093BC
:1037D000CB0108951092CB0108959091CA01892BD5
:1037E0008093CA01089580959091CA01892380939E
:1037F000CA0108951092CA0108958093B9010895ED
:103800001092B901089580910E0190910F01FC0171
:1038100031969C01205F3F4F80E0919191118F5F25
:10382000E217F307D1F70895E0910E01F0910F012F
:103830008091CB018083E0910E01F0910F01908186
:103840008091CA01892B80838091B901882361F01E
:10385000E0910E01F0910F019081892B80830E94ED
:10386000031C81111092B90180910E0190910F01FA
:103870000C94CE10CF92DF92EF92FF926C01EE2467
:10388000FF24C114D104E104F10421F0C701B60101
:1038900020E101C020E0C72ED82EE92EFF24C1145C
:1038A000D104E104F10419F0285FC701B6016B01EE
:1038B0007C0154E0F694E794D794C7945A95D1F7D5
:1038C000C114D104E104F10419F02C5FC701B60161
:1038D0006B017C0142E0F694E794D794C7944A9533
:1038E000D1F7C114D104E104F10419F02E5FC7012E
:1038F000B601DC01CB01B695A79597958795892BE5
:103900008A2B8B2B09F02F5F822FFF90EF90DF9097
:10391000CF9008958091E401843011F120E488E192
:1039200090E00FB6F894A895809360000FBE2093A6
:10393000600083B7817F846083BF83B7816083BF6A
:103940007894889583B78E7F83BF0FB6F894A89537
:1039500080916000886180936000109260000FBECB
:10396000089508950C94B11CCF930E94B21C0E943C
:1039700098060E94B11CC0E08C2F0E948E07811116
:1039800004C0CF5FCE30C1F701C081E0CF91089570
:103990000E942B160E94C2100C94B80982E084BDCC
:1039A00093E095BD9AEF97BD80936E0008952FB771
:1039B000F8948091CD019091CE01A091CF01B0916A
:1039C000D0012FBF0895CF92DF92EF92FF920F9315
:1039D0001F932FB7F8944091CD015091CE01609183
:1039E000CF017091D0012FBF6A017B01EE24FF242B
:1039F0008C0120E030E0C016D106E206F30610F498
:103A0000415051099A01281B390BC9011F910F918F
:103A1000FF90EF90DF90CF9008951F920F920FB616
:103A20000F9211248F939F93AF93BF938091CD01F9
:103A30009091CE01A091CF01B091D0010196A11D2E
:103A4000B11D8093CD019093CE01A093CF01B0938F
:103A5000D001BF91AF919F918F910F900FBE0F90AA
:103A60001F9018950E94BA0DF8942FEF87EA91E6FF
:103A7000215080409040E1F700C0000087E090EBCB
:103A8000DC018093ED019093EE01A093EF01B093E0
:103A9000F0019CE088E10FB6F894A895809360004F
:103AA0000FBE90936000FFCFEF92FF920F931F9392
:103AB000CF93DF93D82FC0E08C2F0E948E0700E0B9
:103AC00010E0E82EF12CC701002E02C095958795D5
:103AD0000A94E2F780FD06C00F5F1F4F0630110504
:103AE00091F709C0602F7C2F80E00E9456088D134B
:103AF000F3CF81E004C0CF5FCE30F1F680E0DF91FC
:103B0000CF911F910F91FF90EF900895CF93C82F01
:103B10008CE20E94541D882321F08C2FCF910C94AD
:103B2000541D80E0CF910895CF930E94DB1E811138
:103B300002C00E94C11EC5E6C15049F00E9498060D
:103B40008FE39CE90197F1F700C00000F5CF89E20F
:103B50000E94861D811113C18AE20E94861D811177
:103B60000E94C11E85E00E94861D81110E94321DA7
:103B70000E94E61E8093CC0187E00E94861D882368
:103B8000A9F18BE10E94861D882351F08091CC0120
:103B900081FB222720F991E0922790FB81F90EC04A
:103BA0008EE00E94861D882361F08091CC0182FB0B
:103BB000222720F991E0922790FB82F98093CC0193
:103BC00015C080E10E94861D9091CC01882341F0B0
:103BD00093FB222720F981E0822780FB93F904C020
:103BE000892F809580FB90F99093CC018091CC0136
:103BF0000E94EA1E0E94F81E8093DE0180EE0E9461
:103C0000861D882341F08091DE01982F909590FBCE
:103C100080F98093DE0189E30E94861D882359F094
:103C20008091DE0181FB222720F991E0922790FB11
:103C300081F98093DE0182EE0E94861D882359F06F
:103C40008091DE0182FB222720F991E0922790FBF0
:103C500082F98093DE0186EE0E94861D882359F04A
:103C60008091DE0183FB222720F991E0922790FBCF
:103C700083F98093DE0183EE0E94861D882359F02C
:103C80008091DE0184FB222720F991E0922790FBAE
:103C900084F98093DE0185E30E94861D882359F014
:103CA0008091DE0185FB222720F991E0922790FB8D
:103CB00085F98093DE0181E30E94861D882359F0F7
:103CC0008091DE0186FB222720F991E0922790FB6C
:103CD00086F98093DE0181E10E94861D882359F0D8
:103CE0008091DE0187FB222720F991E0922790FB4B
:103CF00087F98093DE018091DE010E94FC1E809195
:103D0000DE0187FB882780F980930D0187E20E94FE
:103D1000861DC82F8EE10E94861D8111C2608FE131
:103D20000E94861D8111C46080E20E94861D81115F
:103D3000C86081E20E94861D8111C06182E20E94FA
:103D4000861D8111C06283E20E94861D8111C064BC
:103D500084E20E94861D882311F0C06802C0CC2333
:103D600029F08C2F0E94F31E6C2F03C00E94EF1EBF
:103D7000682F70E080E090E0CF910C94E219CF9131
:103D800008956DEE7EEF80E090E00E94352560E0C2
:103D900082E090E00E94272560E083E090E00E94AE
:103DA000272560E084E090E00E94272560E085E020
:103DB00090E00C94272580E090E00E94212521E0EE
:103DC0008D3E9E4F09F020E0822F089582E090E022
:103DD0000C941925682F82E090E00C94272583E04D
:103DE00090E00C941925682F83E090E00C9427252F
:103DF00084E090E00C941925682F84E090E00C9406
:103E000027258091D30180FF0BC06091130185E0CD
:103E1000689FB001112475956795759567952BC0BE
:103E200081FF09C06091130185E0689FB0011124F2
:103E30007595679520C082FF07C06091130185E0EA
:103E4000689FB001112417C09091D4019923D1F03B
:103E500060911201961788F72091130185E0289F41
:103E600090011124929FA001939F500D112470E0A6
:103E7000CA010E94EB246038710540F46115710598
:103E800019F406C065E070E0862F08958FE7089565
:103E900081E008958091D30180FF08C060911101F5
:103EA00070E0759567957595679521C081FF06C08F
:103EB0006091110170E07595679519C082FF04C08B
:103EC0006091110170E010C09091D401992399F094
:103ED000609110019617A0F780911101899FC00190
:103EE000112470E00E94EB246038710540F46115E4
:103EF000710519F406C061E070E0862F08958FE720
:103F0000089581E00895803F21F40E94011F81956A
:103F100004C0813F29F40E94011F8093D7010895B6
:103F2000823F21F40E94011F819504C0833F29F440
:103F30000E94011F8093D6010895893F19F40E94C1
:103F40004A1F05C08A3F31F40E944A1F8195809321
:103F5000D80108958B3F21F40E944A1F819504C027
:103F60008C3F29F40E944A1F8093D9010895843F11
:103F700021F48091D501816017C0853F21F48091A3
:103F8000D501826011C0863F21F48091D501846003
:103F90000BC0873F21F48091D501886005C0883F20
:103FA00031F48091D50180618093D50108958D3FD2
:103FB00021F48091D30181600BC08E3F21F4809168
:103FC000D301826005C08F3F29F48091D3018460C2
:103FD0008093D3010895803F39F48091D70187FF02
:103FE0006CC01092D70169C0813F29F48091D7013C
:103FF0001816BCF362C09091D601823F29F497FF56
:104000005CC01092D60159C0833F19F41916CCF345
:1040100054C0893F41F48091D80118160CF04DC06E
:104020001092D8014AC08A3F29F48091D80187FFB5
:1040300044C0F6CF8B3F39F48091D90187FF3DC052
:104040001092D9013AC08C3F29F48091D9011816F9
:10405000BCF333C0843F21F48091D5018E7F17C01B
:10406000853F21F48091D5018D7F11C0863F21F4D9
:104070008091D5018B7F0BC0873F21F48091D501C2
:10408000877F05C0883F31F48091D5018F7E809372
:10409000D50113C08D3F21F48091D3018E7F0BC0D9
:1040A0008E3F21F48091D3018D7F05C08F3F29F48D
:1040B0008091D3018B7F8093D3018091D6018111B0
:1040C0000EC08091D70181110AC08091D801811161
:1040D00006C08091D901811102C01092D4010895C7
:1040E00085ED91E00E94D9100E94D71C9093D201D7
:1040F0008093D10108951F93CF93DF938091D101D5
:104100009091D2010E94E31CAC019091D4019923BB
:1041100021F02091140130E006C0209115018AE0C1
:10412000289F900111244217530708F485C08091FD
:10413000D601C091D701D091D8011091D901811138
:1041400007C0C11175C0D11173C0111171C074C005
:104150009F3F19F09F5F9093D401181624F40E949A
:10416000011F8093D6018091D60187FF05C00E9470
:10417000011F81958093D6011C1624F40E94011F13
:104180008093D7018091D70187FF05C00E94011F4E
:1041900081958093D7016091D601662331F1C0915A
:1041A000D701CC2311F1062E000C770B880B990B4D
:1041B0000E94F22323E333E343E35FE30E945624A8
:1041C0000E94BA236093D6016C2FCC0F770B880B1B
:1041D000990B0E94F22323E333E343E35FE30E945E
:1041E00056240E94BA236093D7011D1624F40E941E
:1041F0004A1F8093D8018091D80187FF05C00E9493
:104200004A1F81958093D801111624F40E944A1FF9
:104210008093D9018091D90187FF05C00E944A1F70
:1042200081958093D901DF91CF911F910C947020DB
:104230009F3F09F08FCFA0CFDF91CF911F910895BD
:10424000E5EDF1E085E0DF011D928A95E9F7109236
:10425000D4011092D3010895833081F128F4813084
:1042600059F08230D1F00895853009F449C0B8F191
:10427000863009F456C0089580911501262F30E04C
:10428000280F311D2F3F310524F4680F609315016D
:1042900008958FEF80931501089580911401262FC2
:1042A00030E0280F311D2F3F310524F4680F609353
:1042B000140108958FEF80931401089580911301E4
:1042C000262F30E0280F311D2F3F310524F4680FD1
:1042D0006093130108958FEF8093130108958091E7
:1042E0001201262F30E0280F311D2F3F310524F415
:1042F000680F6093120108958FEF80931201089563
:1043000080911101262F30E0280F311D2F3F3105FC
:1043100024F4680F6093110108958FEF80931101C9
:10432000089580911001262F30E0280F311D2F3F76
:10433000310524F4680F6093100108958FEF809386
:1043400010010895833011F128F4813049F0823052
:1043500091F00895853081F120F18630C1F1089502
:1043600080911501681720F4861B8093150108952C
:1043700010921501089580911401681720F4861B8E
:1043800080931401089510921401089580911301EF
:10439000681720F4861B809313010895109213016F
:1043A000089580911201681720F4861B80931201F2
:1043B000089510921201089580911101681720F458
:1043C000861B809311010895109211010895809128
:1043D0001001681720F4861B809310010895109235
:1043E000100108950F931F938D3109F46BC008F0ED
:1043F0003FC08E3009F47DC0C0F4873009F46EC030
:1044000068F4863009F0AFC08091CC01817F8E7F47
:104410008093CC0181E08093DB01A6C0883009F451
:1044200058C08B3009F49BC09EC0863109F497C0F8
:1044300078F4803109F470C0813109F094C00E9491
:104440002B1690910D0181E0892780930D0187C083
:10445000893109F484C08B3109F085C08091CC0189
:1044600081FB222720F991E0922790FB81F94AC035
:10447000853309F45BC048F4873209F457C008F467
:104480005AC0893209F452C06EC0833438F48A337A
:1044900008F067C0883309F462C065C0833409F44A
:1044A00045C0883409F05FC00E942B160FEF13ED52
:1044B00020E3015010402040E1F700C000000E94BE
:1044C000321D4DC00E9474230E94C2100E94B80980
:1044D00046C00E94E61E0E94F81E41C09091CC0189
:1044E000892F817090FF12C0917F9E7F9093CC01A5
:1044F0003BC08091CC0182FB222720F991E09227DA
:1045000090FB82F98093CC01992349F18091CC01F1
:1045100081608093CC0123C08091CC0183FB222752
:1045200020F991E0922790FB83F9ECCF61E070E0F5
:1045300080E090E010C08D5141E050E060E070E01C
:104540008A019B0104C0000F111F221F331F8A958F
:10455000D2F7C901B8010E94E2190E942B1681E02E
:1045600003C08953E9CF80E01F910F91089580E047
:1045700008950C94B722CF93C82F8091DB0181302E
:1045800079F018F08230E9F187C0E0910E01F091E6
:104590000F018081813169F0823209F07FC009C04A
:1045A000E0910E01F0910F018081813111F0823292
:1045B00061F48C2F0E94B922811104C08C2F0E94BB
:1045C000F2211DC081E090E01AC08C2F0E94B7221A
:1045D000811114C0C43179F048F4CB3079F0C03186
:1045E00009F060C082E08093DB0108C0C93219F095
:1045F000C83321F057C01092DB0154C081E08170B4
:1046000053C0C93289F118F5C43171F1A8F4C7302B
:1046100009F046C08AE08093150194E1909314015B
:1046200093E0909313018093120188E0809311012D
:1046300088E28093100134C0CE51C63088F5EC2F4B
:10464000F0E0E65DFE4F80818093DA0129C0CE3430
:10465000E9F020F4CB3421F56AE013C0C13579F0DC
:10466000C235F1F461E00DC08091DA01882319F0C0
:104670001092DA0115C081E08093DB0115C061E082
:1046800006C08091DA010E942C210AC06AE0809164
:10469000DA010E94A22104C01092DB0180E004C074
:1046A00081E002C080E0ABCFCF910895E1E8F0E077
:1046B0008081886080838081816080838FB7F89457
:1046C00093E09093890090ED909388008FBF0895B8
:1046D000EFE6F0E08081826080830895EFE6F0E00D
:1046E00080818D7F80830895EFE6F0E0908182E005
:1046F0008927808308951F920F920FB60F9211247D
:104700002F933F934F935F936F937F938F939F93D9
:10471000AF93BF93EF93FF938091DC019091DD0104
:1047200001969093DD018093DC01811103C082E04A
:104730000E94B809E091DD01E695E695F0E0E557C5
:10474000F94FE4918091DC018E1303C080E00E9458
:10475000B809FF91EF91BF91AF919F918F917F9198
:104760006F915F914F913F912F910F900FBE0F90DE
:104770001F9018950E94C1236894B1110C94502485
:1047800008950E94352488F09F5798F0B92F9927F3
:10479000B751B0F0E1F0660F771F881F991F1AF02C
:1047A000BA95C9F714C0B13091F00E944F24B1E01E
:1047B00008950C944F24672F782F8827B85F39F01D
:1047C000B93FCCF3869577956795B395D9F73EF4C5
:1047D00090958095709561957F4F8F4F9F4F08956D
:1047E000E89409C097FB3EF490958095709561958B
:1047F0007F4F8F4F9F4F9923A9F0F92F96E9BB2741
:104800009395F695879577956795B795F111F8CFBC
:10481000FAF4BB0F11F460FF1BC06F5F7F4F8F4F27
:104820009F4F16C0882311F096E911C0772321F01D
:104830009EE8872F762F05C0662371F096E8862FB5
:1048400070E060E02AF09A95660F771F881FDAF70C
:10485000880F9695879597F9089557FD9058440FBE
:10486000551F59F05F3F71F04795880F97FB991FCF
:1048700061F09F3F79F0879508951216130614068C
:10488000551FF2CF4695F1DF08C016161706180619
:10489000991FF1CF86957105610508940895E894F4
:1048A000BB2766277727CB0197F908950E946924D3
:1048B0000C94DA240E94CC2438F00E94D32420F0F7
:1048C000952311F00C94C3240C94C92411240C9446
:1048D00050240E942D2470F3959FC1F3950F50E052
:1048E000551F629FF001729FBB27F00DB11D639FA2
:1048F000AA27F00DB11DAA1F649F6627B00DA11D48
:10490000661F829F2227B00DA11D621F739FB00DED
:10491000A11D621F839FA00D611D221F749F33275D
:10492000A00D611D231F849F600D211D822F762FF6
:104930006A2F11249F5750409AF0F1F088234AF0D3
:10494000EE0FFF1FBB1F661F771F881F915050403F
:10495000A9F79E3F510580F00C94C3240C94502479
:104960005F3FE4F3983ED4F3869577956795B795C6
:10497000F795E7959F5FC1F7FE2B880F911D9695E0
:10498000879597F9089597F99F6780E870E060E050
:1049900008959FEF80EC089500240A9416161706D8
:1049A00018060906089500240A9412161306140620
:1049B00005060895092E0394000C11F4882352F083
:1049C000BB0F40F4BF2B11F460FF04C06F5F7F4F3B
:1049D0008F4F9F4F089597FB072E16F4009407D032
:1049E00077FD09D00E94052507FC05D03EF490957F
:1049F00081959F4F0895709561957F4F0895EE0FB3
:104A0000FF1F0590F491E02D0994AA1BBB1B51E1F7
:104A100007C0AA1FBB1FA617B70710F0A61BB70B2E
:104A2000881F991F5A95A9F780959095BC01CD01D3
:104A30000895F999FECF92BD81BDF89A992780B566
:104A40000895A8E1B0E042E050E00C943C25262F08
:104A5000F999FECF1FBA92BD81BD20BD0FB6F89463
:104A6000FA9AF99A0FBE019608950E942725272FDA
:104A70000C942825DC01CB01FC01F999FECF06C07E
:104A8000F2BDE1BDF89A319600B40D92415050400C
:084A9000B8F70895F894FFCF78
:104A98002002B909490A240AF009BC090101BA012E
:104AA80028080A03140A3F4D36394C06FF05C90584
:104AB800900523053C0555056E050102030405060E
:044AC80007080900D2
:00000001FF
